:1005510020493263206C696E6520737461742E20AA
:100561006572722E002053797374656D2052455364
:100571004554002025322E58200025730020537940
:100581007374656D2048414C54454400202E2E2E35
:10059100205361766500202E2E2E2045646974005B
:1005A1002025332E643A0020464C002025322E644B
:1005B10000204578742E204B657970616420657246
:1005C100726F72002042617365202025332E6420F2
:1005D1002D203078255820200020566563746F72D5
:1005E100202025332E64205B78203531325D0020B8
:1005F100456E61626C656420002044697361626CC0
:1006010065640020436F6E6669726D205245434FE9
:100611005244202E2E2E00205265636F7264696E43
:1006210067202E2E2E20002043414E43454C454449
:10063100202E2E2E202000205265636F7264656487
:100641003A2025332E6420736574730020496E644B
:100651006578696E67202E2E2E2000204E6F204473
:100661004D582D35313220646174612020202000E5
:1006710020617661696C61626C65202020202020F8
:10068100202020200020436F6E6669726D20435246
:1006910045415445202E2E2E002050726F63657304
:1006A10073696E67202E2E2E202020200020536596
:1006B1006C65637420566563746F7223202E2E2E31
:1006C1000020496E6372656D656E74202025332E9E
:1006D10064200020436F6E6669726D2052454C4F55
:1006E1004144202E2E2E00202E2E2E204C6F616490
:1006F100656400204C4F47202D2025322E640020B8
:10070100536F6674205265736574202E2E2E00205F
:100711002D2D3E2020506C656173652057616974F1
:100721000062792050454741535553202D203230E6
:100731003031007777772E706567617375732D732C
:1007410079732E6E657400202E2E2E2053656C65F4
:10075100637400202E2E2E20456469742020002011
:100761002E2E2E2043616E63656C20496E70757468
:1007710000444D582D353132205265636F726465E6
:10078100720056312E30302D423231303200286322
:1007910029205045474153555320323030320020F3
:1007A100566572696679696E672052414D202E2E19
:1007B1002E0052414D20636F727275707465640032
:1007C10020526573746F72696E6720646174612071
:1007D1002E2E2E0020566563746F723A205B2532EF
:1007E1002E645D002573202025322E642F25730091
:1007F100257320202D2D2F25730058580025322ECA
:100801006400205858000001020203040505060790
:100811000809090A0B0C0D0D0E0F101011121314FB
:10082100141516171718191A1B1B1C1D1E1E1F2025
:100831002122222324252626272829292A2B2C2D4B
:100841002D2E2F3030313233343435363737383975
:100851003A3B3B3C3D3E3F3F40414242434445469B
:1008610046474849494A4B4C4D4D4E4F50505152C5
:100871005354545556575858595A5B5B5C5D5E5FEB
:100881005F6061626363451959205265636F7264E9
:10089100696E670000000000000000000020506C3D
:1008A10061796261636B20000000000000000000BC
:1008B10000204E6F6E652061747461636865642009
:1008C100000020504C4320313620782031204D75D6
:1008D100780000204B6579626F6172642032207864
:1008E10020380000204C6976652073747265616D53
:1008F100202000204C6F63616C20486561702020CE
:10090100200020566563746F72205B783531325D4B
:10091100004F7065726174696F6E204D6F64652060
:100921000000000000444D582057696E646F772025
:10093100202020200000000000566563746F7220A3
:100941004E756D62657220200000000000496E74D2
:10095100657266616365205479706520000000004E
:1009610000446973706C6179204D6F6465202020AB
:1009710000000000005465726D696E6174696F6EEC
:100981002020202000000000005265636F72642067
:1009910053747265616D202000000000005465737E
:1009A1007420566563746F722020202000000000BF
:1009B100005465737420496E6372656D656E7420B1
:1009C100000000000041636F757374696320626504
:1009D10065702020000000000052656C6F6164208A
:1009E10064656661756C7473000000000045727285
:1009F1006F7220436F646573202020200000000087
:100A010000436F707972696768742020202020206C
:100A110000000000005265636F72640000506C6159
:100A210079626B00004C20004820005620004E6F78
:100A31006E6500566F696400205278440020547836
:070A410044005061737300D3
:0A270C00C10CC10FC10DC10EC110B8
:101489002416F9740A3EFA90426274FFF0A3EAF056
:10149900A3E9F022AF4AEF3395E0EF7F0025E0FEA4
:1014A900EF2432F974003EA801FC7D017B017A002A
:1014B900790022904232E0FBA3E0FAA3E0F9020EA0
:1014C900A3AF4DEF3395E0FE7C0022E475F00102F5
:1014D9000EE0E0FFEE24FAFDE4341FFC227D031246
:1014E9000ECE74262FF9740A3EFA22E4FCFDFEFBA7
:1014F9007A02F9F8020F0CE4FCFDFB7A02F9F8D341
:10150900020F5B74002532F58274003531F58322B0
:10151900E004F0E0C3940522754A01754C01F54DCC
:10152900754E0122AF4BEF3395E0FEEF780322ECC5
:10153900F0A3EDF0A3227B007A007937227B007AB1
:1015490000791622754F00755001227F0025E0FEB3
:02155900EF227F
:10256E001226857F4012266D7BFF7A057951120A5D
:10257E00B37F1412266D7BFF7A057966120AB3D2E9
:0A258E00037FD07E0712237B80FE3E
:10265500D2FFD2FE7F0A7E001224E630FE0530FF4F
:0826650002D32212256EC322EC
:0A18CB0090425BEB121495A3EDF0C0
:1018D5007540FFD20230FF0320FE0FE540600B1577
:1018E500407F327E001224E680EBE540700312252E
:1018F5006EC2FF122720C2FE30024890425EE060B1
:101905004290425B1214BFF53F753E08E53E6013F9
:10191500E53F25E0F53F92FF153ED2FE122720C296
:10192500FE80E9D2FFD2FE122720A2FFB39202C2A7
:10193500FE90425C1214D490425EE014F0D2AED216
:0E194500BE80B5C2FFD2FE122720D2FFA20242
:011953002271
:0A139C0090423CEFF0A3EB12149511
:1013A600753EFFE4F53FF54030FF0320FE0FE53EB6
:1013B600600B153E7F327E001224E680EBE53E7020
:1013C6000312256EC2FF122720C2FE753B08E53BBD
:1013D600601590423CE0FF25E0F092FF153BD2FEFF
:1013E600122720C2FE80E7D2FFD2FE122720A2FFDC
:1013F600B39202C2FE7F327E001224E6300276905D
:101406004240E07002A3E0606CE4F53C753D8075F7
:101416003B08904241E024FFF0904240E034FFF068
:10142600E53B6015D2FE153B30FF04E53D423CC26C
:10143600FEE53DC313F53D80E7904240E07002A310
:10144600E06004C2FF8002D2FFD2FE122720C2FE55
:10145600D2FF90423DE0FBA3E475F001120EF6A91F
:10146600F0FAE53C120EBC0540E5407002053FD29D
:10147600AED2BE8087C2FFD2FE122720D2FFAE3F79
:02148600AF4075
:011488002241
:081AE00090423A121538EBF0B8
:101AE800753A05C201EF249B602C0470567536A028
:101AF80090423BE0F537A3E0F538200146E53A602F
:101B0800427B007A0079367D031218CB92012001BE
:101B1800E9121B4E80E47536A090423AE0F537A3EF
:101B2800E0F538A3E0F539200119E53A60157B00A6
:101B38007A0079367D041218CB92012001E9121B34
:051B48004E80E4A20143
:0B1B4D00227F017E00120026153A22C4
:0B17B600904289121538EAF0A3EBF016
:1017C100751505C211EF249B60340470667510A075
:1017D10090428AE0F51190428CE0F51290428BE044
:1017E100F51320114EE515604A7B007A0079107DD2
:1017F100041218CB92112011E912183780E47510E8
:10180100A0904289E0F511A3E0F51290428CE0F539
:101811001390428BE0F514201119E51560157B003A
:101821007A0079107D051218CB92112011E9121856
:051831003780E4A21164
:0B183600227F017E0012002615152203
:081A600090423AECF0A3EDF016
:101A6800753A05C201EF249B60250470487537A0BC
:101A780090423BE0F53820013CE53A603812153FCA
:101A88007D021218CB92012001EC121AD680E7755C
:101A980037A090423AE0F538A3E0F539200116E581
:101AA8003A601212153F7D031218CB92012001EC07
:101AB800121AD680E730011312153F904240E4F025
:0D1AC800A304F07FA112139CAF37227F0012
:0B1AD500227F017E00120026153A223D
:08169D0090428DECF0A3EDF08A
:1016A500751905C212EF249B60250470487516A0B4
:1016B50090428EE0F51720123CE519603812154668
:1016C5007D021218CB92122012EC12172080E775BA
:1016D50016A090428DE0F517A3E0F518201216E547
:1016E5001960121215467D031218CB92122012ECC6
:1016F50012172080E730121E121546904240E4F082
:10170500A37402F07FA112139CE517FE7C00E4256B
:0A17150016FFEC3EFE227E007F006E
:0B171F00227F017E0012002615192217
:071C3800904234EB121495F9
:101C3F0090425A7405F0C201EF249B7058904237BE
:101C4F0074A0F0ECA3F0A3EDF0E4FFEFC3942050E9
:101C5F001C9042341214BFFE743A2FF582E43442C2
:101C6F00F583EEF00F9042351214D480DE2001255B
:101C7F0090425AE0601F7B017A4279377D23121818
:101C8F00CB92012001E77F017E0012002690425A7D
:071C9F00E014F080D8A2015F
:011CA600221B
:0A160900904233121538EB121495CD
:10161300753705C200EF249B602804704E7534A013
:10162300904234E0F535200042E537603E7B007A96
:101633000079347D021218CB92002000E912169330
:1016430080E47534A0904233E0F535A3E0F536200D
:101653000019E53760157B007A0079347D03121891
:10166300CB92002000E912169380E430001D9042D3
:1016730035E0FBA3E0FAA3E0F9A3E0FFA3E0904287
:0F16830040CFF0A3EFF07FA102139C7E007F0009
:0B169200227F017E0012002615372287
:10229F0075397820940BA20292037F0A7E001223D5
:1022AF007B43E80FD2EED2ECE5E8540FF53830015E
:1022BF001D20941AE539600B7F0A7E001200261547
:1022CF003980EED2037F0A7E0012237B80E3C2EEB9
:0A22DF00C2ECC2C1C20CD2B9AF3884
:0122E90022D2
:1026140075367820941AE536600B7F0A7E00120026
:1026240026153680EED2037F0A7E0012237B80E3D8
:06263400C2C1C20CD2B9C4
:01263A00227D
:0D26E5003094097F017E0012002680F4224F
:081CA700904236EFF0A3EDF0CE
:101CAF00904236E0FF7DF97C1F121A60904238EFA8
:101CBF00F0FE9042361214DBA3E0FB121AE09042C2
:101CCF003812151950028001C34005E4904238F0D4
:101CDF00904236E0FF904238E0FB7DF97C1F121AEC
:101CEF00E0E4904239F0D2037F1E7E0012237B7F07
:101CFF00C87E00120026904239E004F0E0C394063B
:021D0F0040E4AE
:011D110022AF
:05184100904232EFF0BF
:10184600E0FF7DF97C1F121A60904233EFF0E0143E
:10185600F0E4A3F0904233E0C3940550028001C344
:1018660040069042337404F0904232E0FFA3E01247
:1018760014DE121A60904234E02435F582E43442D4
:10188600F583EFF0904233E014F0A312151940C42B
:10189600E4904234F0904234E0FFC3940550257B37
:1018A600FF7A05797474352FF582E43442F583E0C6
:1018B600FF904262E4F0A3EFF0120AB3904234E0E4
:0418C60004F080D1D9
:0118CA0022FB
:0524B300904232EFF041
:1024B800E0FFE4FB7DF97C1F121AE0E4904233F060
:1024C800904233E0FEC3940550139042321214DB5D
:0D24D8007BFF121AE0904233E004F080E335
:0124E50022D4
:1022EA00904232EFF0A3EB1214951226857F40122A
:1022FA00266D904233E0F9A3E0FAA3E0904262C966
:10230A001214957BFF7A05797B120AB37F14122681
:10231A006D7BFF7A05797E120AB3904232E0FF7D27
:0A232A00F2121CA7D2AED2BE80FA58
:1026B10020010F12154DE4F54B12152175480175D6
:0326C100490122AA
:1026C400E4F54BF54F755001121521754901F54894
:0126D40022E3
:1025EC007F5412266D7BFF7A05798D120AB3D201C6
:1025FC001226B17FF47E011200267F5412266D7BC9
:08260C00FF7A057997020AB379
:0D26F20075988075A910C298C299D29B22DC
:07195400904232EB121495E2
:10195B007F4012266D7BFF7A0579A1904262E54F9D
:10196B00F0A3E550F0120AB3E4904235F090423503
:10197B00E0FFC394035057EF90088793FF12266D37
:10198B00E4904236F01214BCB4FF0B7BFF7A05795E
:10199B00A8120AB3801E1214BCFFC313900807933E
:1019AB00FE3395E0904262F0A3CEF07BFF7A05798F
:1019BB00AC120AB39042331214D4D2AED2BE9042C0
:0E19CB003612151940BF904235E004F0809F9F
:0119D90022EB
:051E4800904233EFF0B1
:101E4D00E0FF1214F48E388F39E4F53AF53B9042E9
:101E5D0033E0B41F05753D0F8003753D10E4F53C6F
:101E6D00E53CC3953D50367400253BF97400353A79
:101E7D00FA7B01AD39AC387F65121C387F0A7E00C4
:101E8D00120026053C74202539F539E43538F5382E
:0D1E9D007420253BF53BE4353AF53A80C34F
:011EAA002215
:10243F00753705C200EF5407FF25E0447154FEF5D0
:10244F0034AF058F3520001FE537601B7B007A0006
:10245F0079347D021218CB92002000E97F017E00B3
:09246F00120026153780DEA200E0
:012478002241
:10000300EF5407FF25E04471FF7B007A00793490B9
:0C0013004240E4F0A304F012139CAF3450
:01001F0022BE
:0723C000904232EB1214956C
:1023C700C2AFD29BC2B1753450D534FDD2B175348A
:1023D7000CD534FDE4F5993099FDED4C601C904225
:1023E700321214BFF5993099FD9042331214D4ED8F
:0C23F7001D70011CD2AED2BE80E0D2AF3F
:0124030022B6
:03002000D2B12238
:102515001226857F4012266D7BFF7A0579B2120A55
:10252500B37F1412266D7BFF7A05797E120AB3D22A
:0E253500037FD07E0712237BD2AED2BE80FA87
:101EAB00753905C200EF54FEF534753580753681F2
:101EBB00753782E53525362537F538200035E53978
:101ECB0060317B007A0079347D051218CB400BD240
:101EDB00037F327E0012237B80157F907E011224BC
:101EEB00E620FE04D20080077F327E00120026150A
:101EFB003980C87F147E00120026E5396002D32298
:011F0B00C312
:011F0C0022B2
:10203200753805C200EF54FEF534753561AF058F72
:1020420036E5352536F537200035E53860317B0039
:102052007A0079347D041218CB400BD2037F327E92
:102062000012237B80157F907E011224E620FE045D
:10207200D20080077F327E00120026153880C87F8A
:0D208200057E00120026E5386002D322C35F
:01208F00222E
:10209000753805C200EF54FEF534753560AF058F15
:1020A00036E5352536F537200035E53860317B00DB
:1020B0007A0079347D041218CB400BD2037F327E34
:1020C0000012237B80157F907E011224E620FE04FF
:1020D000D20080077F327E00120026153880C87F2C
:0D20E000057E00120026E5386002D322C301
:0120ED0022D0
:1020EE00753C05C201EF54FEF538753962AF058FA8
:1020FE003AE539253AF53B200135E53C60317B0068
:10210E007A0079387D041218CB400BD2037F327ED1
:10211E000012237B80157F907E011224E620FE04A0
:10212E00D20180077F327E00120026153C80C87FC8
:0D213E00057E00120026E53C6002D322C39E
:01214B002271
:0521A600904232EFF051
:1021AB00753505E4A3F0A3F0904233E0FEA3E0FF06
:1021BB00E4FCFD7B01FAF9F8C3120F5B6027E535F0
:1021CB006023904232E04401FF1B7A007934904245
:1021DB0040E4F0A304F012139C904233EEF0A3EF13
:0E21EB00F0153580C3E5356003AF34227FFF69
:0121F90022C3
:03002300021F0DAC
:101F0D00C0E0C0D075D008309A38300F4C300D106D
:101F1D00E5996007755401C20F8005755402C20D15
:101F2D00E5524551600AE5521552702D1551802923
:101F3D0074552553F8A6990553E553B4101BC20FDC
:101F4D008017E599700E854F51855052F553D20D7E
:101F5D00D20F8005C20F75540AC298C299D0D0D045
:021F6D00E03260
:03004B0002271772
:05271700D20CC2B93232
:101D1200C200D201A200920212229F8F36EF640209
:101D22006055E536B4040E154BC3E54B64809480D0
:101D32005003754B01E536B4080E054BD3E54B64F1
:101D42008094814003E4F54BE536B401031225EC9F
:101D52007F4012266DAF4B1214CC7D14120ECE743E
:101D62008A2FF974083EFA7BFF120AB3E54924FF71
:071D720092001226E5809BA0
:011D79002247
:1019DA00C201C20212229F8F36EF6402606BE536A3
:1019EA00B404140550E5507002054FD394F2E54F44
:1019FA009401400312154DE536B40819E550155007
:101A0A007002154FC3E5509401E54F9400500675D6
:101A1A004F017550F2E536B401031225EC7F4012EE
:101A2A00266D7BFF7A0579C5904262E54FF0A3E502
:101A3A0050F0FFA3E54FF0A3EFF0120AB37FC87E80
:101A4A00001200261226E58087E54924FF92037FCB
:061A5A000A7E0002237B5E
:101B5800C201C20212229F8F36EF64026055E53639
:101B6800B4040E054AD3E54A648094A04003754A3C
:101B780001E536B4080E154AC3E54A6480948150DD
:101B880003754A20E536B401031225EC7F4012267E
:101B98006D7BFF7A0579DAAF4AEF3395E0904262C0
:101BA800F0A3EFF0120AB37FC87E001200261226B7
:101BB800E5809DE54924FF92037F0A7E0002237B8E
:101D7A00C200D201A200920212229F8F36EF6402A1
:101D8A006055E536B4040E154CC3E54C6480948066
:101D9A005003E4F54CE536B4080E054CD3E54C6423
:101DAA008094824003754C02E536B401031225EC97
:101DBA007F4012266DAF4C1214CC7D11120ECE74D8
:101DCA00B22FF974083EFA7BFF120AB3E54924FFE1
:071DDA0092001226E5809B38
:011DE10022DF
:101DE200C200D201A200920212229F8F36EF640239
:101DF2006053E536B4040E154DC3E54D64809480FE
:101E02005003754D02E536B4080E054DD3E54D6419
:101E12008094824003E4F54DE536B401031225ECCB
:101E22007F4012266D1214CA7D0F120ECE74E52F5A
:101E3200F974083EFA7BFF120AB3E54924FF9200C7
:051E42001226E5809D61
:011E47002278
:101FD100C200D201A200920212229F8F36EF640248
:101FE100604EE53664046005E536B4080CE54870DA
:101FF100047F0180027F008F48E536B4010312257A
:10200100ECE54824FFB392FC7F4012266DE5486061
:102011000B7BFF7A0579F0120AB380097BFF7A0501
:1020210079FA120AB3E54924FF92001226E580A24B
:01203100228C
:10127200C200E4F536F537200E131213817A06798F
:1012820004120AB3E54924FF92001226E5200E114A
:10129200D201A200920212229FEF640160030213A4
:1012A2007E1226857D087F501220EEE5546402608E
:1012B2000302134D1213817A067918120AB3C2AFD0
:1012C200C298209806D2AED2BE80F7209AF2C29877
:1012D200209806D2AED2BE80F7E5997027309A2EBA
:1012E200C298209806D2AED2BE80F774002537F598
:1012F2008274003536F583E599F00537E53770DD00
:10130200053680D91213897A067928120AB3121384
:10131200897A067938E53724FF904263F0E536345E
:10132200FF904262F01213917A06794D120AB312BB
:10133200149D7E02120E7DE54A14FF121E48C20F52
:101342007FE87E03120026D2AF80157F4012266D01
:101352007BFF7A06795C1213917A067971120AB3CD
:101362007FE87E031200267D147F021224797D1409
:0E1372007F031224797D647F501220EEC20E9C
:10138000227F4012266D7BFF227F4012266D7BFF5D
:0C13900022120AB37F1412266D7BFF228C
:10155B00C200E4904232F0E54A70030215EB12161A
:10156B00017A067986120AB3E54924FF9200122606
:10157B00E5D201A200920212229FEF640170761253
:10158B0016017A06799A120AB3E4F536F537AE36B8
:10159B00AF371215004024904232E0FF740025371C
:1015AB00F58274003536F583EFF00537E5377002B9
:1015BB000536904232E0254EF080D3D2AED2BE1229
:1015CB00149D7E02120E7DD2AED2BEE54A14FF12DE
:1015DB001E487FF47E011200267D147F03022479BE
:1015EB007F4012266D7BFF7A0679AE120AB37FE835
:0515FB007E0312002632
:09160000227F4012266D7BFF22BF
:101BC800C201C20212229F8F36EF64026055E536C9
:101BD800B4040E054ED3E54E648094A04003754EC0
:101BE80020E536B4080E154EC3E54E648094805047
:101BF80003E4F54EE536B401031225EC7F401226C6
:101C08006D7BFF7A0679C2AF4EEF3395E090426262
:101C1800F0A3EFF0120AB37FC87E00120026122646
:101C2800E5809DE54924FF92037F0A7E0002237B1D
:10214C00C200D201A200920212229F8F36EF6402CB
:10215C006047E53664046005E536B4080CE5497063
:10216C00047F0180027F008F49E536B401031225FC
:10217C00EC7F4012266DE549600B7BFF7A0579F008
:10218C00120AB380097BFF7A0579FA120AB3E54982
:09219C0024FF92001226E580A93F
:0121A5002217
:10224E00C2007F4012266D7BFF7A0679D4120AB344
:10225E00E54924FF92001226E5D201A20092021255
:10226E00229FEF640170291226C4D2011226B17F7B
:10227E00F47E011200267F5412266D7BFF7A0679BA
:10228E00E8120AB37F651224B37D147F04122479F9
:01229E00221D
:1021FA00C2007D147F04122479D201A20092021235
:10220A00229F8F36EF640260347F4012266D7DF97B
:10221A007C1F7F65121A60904262E4F0A3EFF07BA4
:10222A00FF7A0679F4120AB37F1412266D7F6512BB
:10223A001841E54924FF92001226E580BC7D147FEF
:04224A0003022479EE
:10254300122685E4FF12266D7BFF7A077900120AB3
:10255300B37F1412266D7BFF7A077910120AB31228
:0B25630026147DF07F65121CA780FE8F
:10233400C200D201A200920212229F8F36EF6402E1
:1023440060277F4012266D7BFF7A077922120AB339
:102354007F5412266D7BFF7A077934120AB3E5495C
:1023640024FF92001226E580C97D147F031224798C
:072374007D147F04022479AF
:10101000E4F5341226851211121211321226E5D28D
:1010200001E54924FF920212229F8F35EF6402707E
:101030000302110BE535B4080A0534E534B40D0399
:10104000E4F534E535B4040E1534C3E53464809416
:1010500080500375340CE535640160030211027F92
:101060005412266D7BFF7A077954120AB3E534B423
:101070000D00506F90107BF82828730210A2021008
:10108000A70210AC0210B10210B60210BB0210C0D1
:101090000210C50210CA0210CF0210D40210D902E9
:1010A00010DE121D1280511219DA804C121B58806A
:1010B00047121D7A8042121DE2803D121FD18038F6
:1010C000121272803312155B802E121BC8802912F7
:1010D000214C802412224E801F1221FA801A1223E2
:1010E0003480157F4012266D7BFF7A077960120AE3
:1010F000B37F207E031200267D147F021224791212
:1011000011321211121226E502101F7D147F040203
:02111000247940
:10111200E4FF12266DAF34EF3395E0FE7C007D14C0
:10112200120ECE74122FF974093EFA7BFF020AB333
:101132007F5412266D7BFF7A077948120AB3022682
:011142001498
:10004E00E4F523F525F526F527F5287529FF752AFC
:10005E00FF752BFF752CFF752DFF752EFFC233F527
:10006E0087F5D01226551226F2D2BED29712002054
:10007E00C2011226B1E4F554FE7F10FDFB7A007921
:10008E0055120F71D2ACD2B9C2CDD200121F6FE48D
:10009E00FF12266D7BFF7A077972120AB37F49121F
:1000AE00266D7BFF7A077983120AB37F5812266D6D
:1000BE007BFF7A07798F120AB31205187FC47E0967
:1000CE001200261226857D057C007F2C7E011211E2
:1000DE00437F4012266D7BFF7A0779A0120AB3E4A4
:1000EE00F531F532AE31AF32121500401A12150C41
:1000FE0074AAF012150CE064AA6002D2330532E540
:10010E003270E1053180DD30330B7BFF7A0779B336
:10011E007F651222EA7E027F007D001214B5120F57
:10012E00717F207E031200267F4012266D7BFF7AA0
:10013E000779C1120AB3E4F5307F1412266D7BFFE6
:10014E007A0779D5E5302401904263F0E43390428A
:10015E0062F0120AB3AF301214F4AD07AC06E530FC
:10016E001215542432F974023EFA7B01904238740F
:10017E0002F0A3E4F07F651216097F0A7E001200DA
:10018E00260530E530C3942040AF7F50121EAB40A1
:10019E0003122515122685D2AFD29CD2AED2BEE561
:1001AE0027700C7527FFF526F525C200121F6FE587
:1001BE00266003020261752608FF12266DE54A606D
:1001CE002F1214CA1214E690426712149312152DB0
:1001DE00C333CE33CED8F9121489AF4AEF3395E03C
:1001EE00A3F0A3EFF07BFF7A0779E5120AB3802222
:1001FE001214CA1214E690426512149312152DC3EE
:10020E0033CE33CED8F91214897BFF7A0779F112E7
:10021E000AB3E54D146012146014240270357B008D
:10022E007A007955121954802A1205218025E54A43
:10023E00601EFF3395E0EF1215542431F974003E21
:10024E00FA7B01E92550F9EA354FFA121954800369
:10025E00120521D2AED2BE309123E54B6401601D52
:10026E00754B01754D017D017F50122032752BFFAC
:10027E00752DFF7529FFE4FD7F501220EE2091129F
:10028E00E54B600EE4F54BF54DFD7F5012203275B7
:10029E002BFFE54B64017032E529654A602C854AD7
:1002AE0029E52960191215542432F974003EFA7B9F
:1002BE000178007C007D017E02120E7D800C7E0294
:1002CE007F007D001214B5120F71E54B7039E529D0
:1002DE00654A6033E54A6022652A6003752F1475FE
:1002EE0029FF854A2AE52F6004152F801A854A2991
:1002FE00752AFFD20E121272800D854A29752AFFB9
:10030E00E4FD7F501220EE200C063094030203D33E
:10031E00120518C201C20212229F8F23E523146018
:10032E002024FD602524FE606824FE604224FE60C9
:10033E007B240760030203D312050D12254302032B
:10034E00D312050D1210100203D3D297C374059564
:10035E0050E4954F500E74FB2550F55074FF354FF9
:10036E00F54F8006754F017550F21205478056D233
:10037E0097D374EC95507401954F400D740525502C
:10038E00F550E4354FF54F800312154D1205478099
:10039E003412053CD3E54A6480F87420648098409A
:1003AE0002054A7F2C7E01120026801912053CC3DD
:1003BE00E54A6480F874016480985002154A7F2CD7
:1003CE007E01120026D2AED2BEE52860030204885A
:1003DE007F0D12266D7F501221A68F30EFD3942001
:1003EE00400B7BFF7A0779FB120AB3801D7BFF7AE5
:1003FE000779FE120530E52E6530600EAF308F4A5C
:10040E008F2ED2001226D57524FA7F011200038F8B
:10041E0030EFD39420400B7BFF7A087903120AB396
:10042E00801D7BFF7A0579AC120530E52C653060B6
:10043E000EAF308F4A8F2CD2001226D57524FA7F3C
:10044E000A7E00120026E52D654A600A854A2DAD0A
:10045E004A7F50122090E52B654A601B854A2BE59A
:10046E004BB4010CE54A4480FDE4FF12243F8007A3
:10047E00AD4AE4FF12243F752805D2AED2BEE54B3D
:10048E00146009047019D2FDD2FC8013C2FDE54838
:10049E0024FFB392FC1214B57D007C021223C0D24D
:1004AE00AED2BEE525702C75251E7F5412266DE545
:1004BE004BB40103755403E55475F005A4242FF9CC
:1004CE00740A35F012148F7BFF7A05797B120AB30A
:1004DE00E4F5541527152615251528D2AED2BEE5FE
:1004EE0024600415248005C2001226D5B297E52695
:0F04FE0070030201A97F3C7E001200260201A9B3
:10050D00D297D2037F0A7E0002237BD2001226D51A
:10051D007524FA2274FF2550F974FF354FFA7B01CB
:10052D00021954904262E4F0A3E530F0020AB3D20E
:10053D0097D2037F0A7E0002237B7526017F647E9E
:04054D000002002682
:10002600E4F542EF4E601DEF1F70011E754166E557
:1000360041600B1541E542F5F0A4F54280F1D2AEE0
:04004600D2BE80DFC7
:01004A002293
:1024E600AD07AC06ED4C6026ED7803CEC313CE13D4
:1024F600D8F9FDAC067802CEC313CE13D8F92DFD5C
:0F250600EE3CFCED4C6007ED1D70F81C80F522DB
:02272000002295
:102598009042347401F0A374F4F0904232E0FEA348
:1025A800E022F0EE904232F022F0904234E0FEA3B6
:0A25B800E0FF22904234E4F0A32279
:10237B0090425FEEF0A3EFF0300339D2ECC2EEE007
:10238B0025E0F090425FE033F090425FE07002A3F3
:10239B00E0601D904260E024FFF090425FE034FF6C
:1023AB00F07FF47E011224E6B2EBD2AED2BE80D91E
:0523BB00C2ECC2EB22A0
:10114300904232EEF0A3EFF0A3ECF0A3ED1225B141
:10115300EE6003021235EFB408004003021235902B
:101163001169F828287302118102119C0211B4023B
:1011730011C10211DB0211ED02120302121F904290
:10118300347427F0A374101225A17802CEC313CEB2
:1011930013D8F91225AA0212449042347413F0A30F
:1011A3007488F0904232E0C313F0A3E013F002120C
:1011B300449042347409F0A374C4F0021244904280
:1011C300347403F0A374E8F0904233E025E0F09028
:1011D3004232E033F00212441225987802C333CE30
:1011E30033CED8F91225AA0212441225BB74FA127F
:1011F30025A17803C333CE33CED8F91225AA804173
:101203001225BB747DF0904233E0C4F8540FC868D4
:10121300F0904232E0C454F048F080251225BB74AC
:101223003E1225A17805C333CE33CED8F91225AAB1
:10123300800F1225987802C333CE33CED8F9122506
:10124300AAD2ECC2EE904232E07002A3E0601B909F
:101253004233E024FFF0904232E034FF1225B11212
:0F12630024E6B2EBD2AED2BE80DBC2ECC2EB22ED
:04271C000040145411
:0D26FF00D2EDD2EDC2ED7F147E000224E684
:102404007546FF85E84743E80FC2ECC2EFD2EED22F
:10241400ED7F287E001224E630EB13E546600F15AD
:10242400467F147E001224E6D2AED2BE80EAC2ED0C
:0A2434008547E8E5466002D322C3A5
:01243E00227B
:1025C200904288EFF0C2EC12240453E8F090428863
:1025D200E0FFC4540F540F42E81226FF53E8F09074
:0A25E2004288E0540F42E80226FF91
:10266D0090425FEFF0C2EC122404C2EFC2EE904232
:08267D005FE04480FF0225C26A
:10263B0090428FEFF0C2EC122404C2EFC2EE904234
:0A264B008FE04440547FFF0225C2D7
:101F6F00E4F5E83000087F14FE12002680077F0199
:101F7F007E0012002675E8031226FF7F057E0012F1
:101F8F000026121FC4121FC475E8021226FF7F011C
:101F9F007E001200267F281225C27F0C1225C27FD9
:101FAF00061225C27F011225C27F021225C27F02AF
:101FBF007E0002002675E8031226FF7F017E0002D5
:021FCF000026EA
:102685007F011225C27F027E001200267F021225DD
:06269500C2E4FF02266D05
:10269B00904287EFF0D2EFC2EEE0FF1225C2C2EFFD
:0626AB00904287E0FF22CF
:10247900904233EFF0A3EDF012249A904234E060D9
:102489000D14F07F2012269BD2AED2BE80ED02241D
:102499009A904233E0FF3395E0FE741B2FF5827466
:0A24A900273EF583E493FF02266D41
:1026D500300004C2968002D2967F017E0002002659
:0300000002172ABA
:0C172A00787FE4F6D8FD75816402177129
:100DAD00E709F608DFFA8046E709F208DFFA803E28
:100DBD0088828C83E709F0A3DFFA8032E309F60815
:100DCD00DFFA8078E309F208DFFA807088828C837D
:100DDD00E309F0A3DFFA806489828A83E0A3F60831
:100DED00DFFA805889828A83E0A3F208DFFA804C0B
:100DFD0080D280FA80C680D4806980F280338010E2
:100E0D0080A680EA809A80A880DA80E280CA80334A
:100E1D0089828A83ECFAE493A3C8C582C8CCC583C2
:100E2D00CCF0A3C8C582C8CCC583CCDFE9DEE78092
:100E3D000D89828A83E493A3F608DFF9ECFAA9F011
:100E4D00EDFB2289828A83ECFAE0A3C8C582C8CC67
:100E5D00C583CCF0A3C8C582C8CCC583CCDFEADE80
:100E6D00E880DB89828A83E493A3F208DFF980CCE2
:100E7D0088F0EF60010E4E60C388F0ED2402B404DB
:100E8D000050B9F582EB2402B4040050AF23234582
:060E9D008223900DFD739D
:100EA300BB010689828A83E0225002E722BBFE024D
:090EB300E32289828A83E4932280
:100EBC00BB010689828A83F0225002F722BBFE0115
:020ECC00F3220F
:100ECE00EF8DF0A4A8F0CF8CF0A428CE8DF0A42E38
:020EDE00FE22F2
:100EE000C5F0F8A3E028F0C5F0F8E582158270029D
:060EF0001583E038F0223A
:100EF600A3F8E0C5F025F0F0E582158270021583AF
:060F0600E0C838F0E8220B
:100F0C00E88FF0A4CC8BF0A42CFCE98EF0A42CFC84
:100F1C008AF0EDA42CFCEA8EF0A4CDA8F08BF0A402
:100F2C002DCC3825F0FDE98FF0A42CCD35F0FCEB61
:100F3C008EF0A4FEA9F0EB8FF0A4CFC5F02ECD3926
:0F0F4C00FEE43CFCEAA42DCE35F0FDE43CFC2293
:100F5B00EB9FF5F0EA9E42F0E99D42F0EC6480C80D
:060F6B0064809845F022AD
:100A4800E5412462F582E43442F583E005412290D1
:100A5800425F300A03904262E475F001120FCA0245
:100A68000EA32003E97F2ED2038018EF540F2490A1
:100A7800D43440D4FF30070BEF24BFB41A0050031E
:100A88002461FFE542600215420545E5457002050F
:100A980044300A0E90425FE475F001120FCAEF026B
:100AA8000EBC02269B7403D20A8003E4C20AF541F5
:100AB80090425F120FE1E4F542F544F545E54260E6
:100AC800077F20120A8B80F57543FFC204C203C258
:100AD80005C206C208C209C20B120A57FF700D30C0
:100AE8000A057F00120A9CAF45AE4422B4255FC2B6
:100AF800D5C207120A57FF24D0B40A00501A75F05D
:100B08000A784230D50508B6FF0106C6A426F620A5
:100B1800D5047002D20680D924CFB41A00EF50044D
:100B2800C2E5D207020C9DD20480C6D20380C0D28F
:100B38000580BCD2D580BAD20880B47F20120A8B37
:100B48002005077401B5420040F1120A48FF120A55
:100B58008B020AC5D20BD2098095120A48FB120AE9
:100B680048FA120A48F94A4B7006796E7A0D7BFFEB
:100B780020052EE542602A7E008E82758300120FC2
:100B88009D60060EEE654370F0C2D5EBC0E0EAC08A
:100B9800E0E9C0E0EE120CE4D0E0F9D0E0FAD0E0F1
:100BA800FB120EA3FF60AAEBC0E0EAC0E0E9C0E0D8
:100BB800120A8BD0E02401F9D0E03400FAD0E0FB2F
:100BC800E5430460DCD543D980877BFF7A0C79E064
:100BD800D205809C791080027908C209C20B80086E
:100BE800D2D5790A8004790AC2D5E543047002F5A2
:100BF80043E4FAFDFEFF120A48FC7B0820041312A6
:100C08000A48FD7B1030030A120A48FE120A48FF00
:100C18007B20EC3382D592D55013C3E43003069F72
:100C2800FFE49EFEE42004039DFDE49CFCE4CBF875
:100C3800C204EC700CCFCECDCCE824F8F870F38069
:100C480017C3EF33FFEE33FEED33FDEC33FCEB332C
:100C5800FB994002FB0FD8E9EB300405F8D0E0C45B
:100C680048B204C0E00AEC4D4E4F78207B0070C2B9
:100C7800EAB5430040BCC0E0120CE6D0F0D0E0205A
:100C88000404C4C0E0C4B204C0F0120A74D0F0D5A1
:100C9800F0EB020AC5120FEA0B62530BDC580B3358
:100CA8004C0B2F420BE04F0BE8440BE8490B484331
:100CB8000BEE550BD2460BD2450BD2470D8E500B7F
:100CC800372D0B3B2E0B5E2B0B3F230B5C200D7C33
:100CD8002A0AF74800000B563F3F3F00790AA2D581
:100CE800200614300809B910020404B9080104A246
:0E0CF800D52009025001042005689205B5427E
:100D0600005034C0E07F203006197F30A2057209FA
:100D16007208500F120D3DC205C209C208C20B7FF0
:100D260030800F300803E9C0E0120A8B300803D088
:100D3600E0F9D0E0B542CC3008177F30B9100C127C
:100D46000A8B7F583007077F788003B90803120A99
:100D56008B3005057F2D020A8B7F20200BF87F2B19
:100D66002009F322920580CF286E756C6C29002D20
:100D760050434958D204120A483004F8C204784253
:100D860030D50108F6020AF7120A482403B4050012
:100D96004001E4900D7593120A7C743A120A7CD2D3
:070DA60006754204020BDC9C
:100F7100EF4E6012EF60010EEDBB010B89828A8397
:100F8100F0A3DFFCDEFA2289F05007F709DFFCA9A4
:0C0F9100F022BBFEFCF309DFFCA9F022FB
:1017360002004EE493A3F8E493A34003F68001F27B
:1017460008DFF48029E493A3F85407240CC8C333B4
:10175600C4540F4420C8834004F456800146F6DF83
:10176600E4800B010204081020408090270CE47EE0
:10177600019360BCA3FF543F30E509541FFEE49378
:10178600A360010ECF54C025E060A840B8E493A33F
:10179600FAE493A3F8E493A3C8C582C8CAC583CA6A
:1017A600F0A3C8C582C8CAC583CADFE9DEE780BE22
:0127160000C2
:100F9D00BB010CE58229F582E5833AF583E0225009
:100FAD0006E92582F8E622BBFE06E92582F8E22253
:0D0FBD00E58229F582E5833AF583E493226D
:100FCA00F8E0FBA3A3E0F925F0F0E58215827002B0
:070FDA001583E0FA38F02254
:090FE100EBF0A3EAF0A3E9F02211
:100FEA00D083D082F8E4937012740193700DA3A396
:100FFA0093F8740193F5828883E4737402936860AA
:06100A00EFA3A3A380DFA9
:00000001FF
